:100000000C94E5031895189518951895189518955A
:1000100018951895189518950C940C021895189524
:10002000189518950C94F001189518951895189531
:100030000C94B40118951895189518950C94820194
:100040001895189518951895189518951895189548
:100050001895189518951895189518951895189538
:100060001895189518951895189518951895189528
:10007000E199FECF1FBB0EBBE09A0DB308950E941D
:100080000C04C801A22F17D0A01739F0F8949FBB19
:100090008EBBADBBE29AE19A7894E3E00C94150430
:1000A0000E940C04C80107D0A02F01968C0103D038
:1000B000102F0A2FF2CFDCCF41D0D801932F19D0C7
:1000C000292F11968D0132C039D0C801A0916B0241
:1000D000B0E0AF73AA0FAA0F1896980108D09C0140
:1000E000129605D020916B0202E010E01FC08D0136
:1000F000E3CFC5CF23D002E010E0DDDF00936B0239
:10010000802F90E08F73880F880F089613D08C0192
:100110000E5F1F4FC5DFA017B10731F022D103AD2D
:100120000A9503AF029706D08D0101C0E2DFE4E03B
:100130000C9414048C01B4DFD80108950C940B04C2
:10014000DC9A03E00A95F1F70000DC9808951BB3F0
:10015000107F02950F70102B1BBBF2CF8A93802F5C
:10016000112311F0DD9A01C0DD981BD08295807FAC
:10017000082F17D00AEF00000A95E9F78991089532
:1001800010E0ECCF11E0FDCFBA93AA93D80101C0E3
:10019000B2D00D910023E1F7A991B991089501D052
:1001A00001C0D5CF03ED10E301501040E9F700C0C6
:1001B00000000895F7DF16D015D014D000E2EFDF6D
:1001C00008E20FD00CE00DD001E00BD0EBDF00E82F
:1001D00008D000EB11E0D8DF00EC03D004EB11E015
:1001E000D3CFCECF00E3DBCF0E9407042897E1D224
:1001F0005888498890E083E0A0EEB1E076D038F5E9
:10020000552081F000E010E020E030E040E050E0D8
:1002100060EF7FE3BED2CDD285E004C0A8EEB1E0AE
:10022000C7D2839564D0A0EFB1E00E944407B0F339
:100230005ED0A8EEB1E059D028F4A0EEB1E0B8D27B
:100240008A95F6CF54D04FD050F456D0FBCF988338
:1002500099839A839B839C839D839E839F8307E0DE
:10026000401669F444D0A8E0B2E0A1D1A2D23BD0BC
:1002700030F492D241D0933014F08A9590E0662405
:1002800019C035D00E94E204A02F005D34D0691659
:1002900011F40EE230D00A2F1A2F110F110B212F5B
:1002A000312F0E94CF04DE010E940506A8EFB1E0C5
:1002B0007FD26394762C770C7708552464147504E8
:1002C00004F318D0982F990F990B880F991F880F56
:1002D000991F08EB11E0080F191F56DF0BD0289665
:1002E000EAE00C941004A8EFB1E00C946A0754D231
:1002F0007F81089500E246CFA0E0B2E048D259D213
:100300009395089528D006A517A57CD006A717A712
:10031000789404A515A576D004A715A704AD039578
:1003200004AF093120F000E004AF01E004AB05A9FF
:10033000002329F005A90A9505AB959A01C0959867
:1003400006A9002329F006A90A9506AB969A01C0D2
:1003500096985BD01895FA93EA932A931A930A9386
:100360002FB7E0E3F2E00895FA93EA934A933A93C1
:100370002A931A930A934FB7F4DF00A111A122A187
:1003800033A126D003A9013091F400A1048B158B71
:10039000268B378B04B515B504A315A306A517A5A1
:1003A00006A317A308B707FD4BD002E003AB08B7BD
:1003B00003FF05C000A111A10BD008E008BF4FBF8B
:1003C00009911991299139914991E991F9911895DA
:1003D00019D02F4F3F4F00A311A322A333A3089599
:1003E000BADF00A911A90ED000AB11AB789407A910
:1003F000039507AB07A90A3F20F000E007AB01E037
:1004000000AFA7CF0F5F1F4F08952FBF099119911C
:100410002991E991F99108959EDF00918000109152
:10042000810000A711A700A911A902A713A7009195
:100430007C0002FD05D001E001AF00E007AB89CFF1
:1004400004A115A10030104828F406A117A1DADF95
:1004500006A317A3089572DE00916802002319F124
:1004600000E00093680200937C0200E010E04091FD
:100470007C0254E0459FF001E358FD4F0083018367
:1004800002830383EDE6F2E08DD078F317871687B9
:1004900010871187128713871093660214871587B8
:1004A00002E300936A0200916902002309F479C013
:1004B00000E0009369028DE692E053DF62A573A528
:1004C00000A511A5FC01008311836283738358D1B9
:1004D000041B150B260B370B408151816281738100
:1004E0003FD1A801B901415C5D41644F70404F3775
:1004F0005C406040704008F054C0478554E0459F20
:10050000ADE7B2E0A00DB11D4085518562857385D0
:10051000FD01008011802280338040195109620959
:100520007309400F511F621F731FFC0140875187E1
:1005300062877387FD0119D1FC0134D010F000E00F
:1005400007870685039506870A3040F10AE006878B
:100550008A019B01F8D0A8EFB1E01CD102DFF5D0F1
:10056000EAEFE0936602FC01A485B5851196A487A5
:10057000B58704841584E8E50E16E2E01E0688F0CF
:10058000A0E0EDE6A487A587A0E1B2E010D0A8E145
:10059000B2E0FDD00E94E20497DD03C003E50093C2
:1005A0006602C5CD0785039507870A3008950C9428
:1005B0007105289701E007B908E002BB0FE30ABB09
:1005C00000EE01BB07E003BFF5DD80E392E092DDC2
:1005D000212F220F220B322F0E94CF04EAD0DCD031
:1005E000A8E1B2E0D7D0A0E2B2E0E1DFFC01ADD0FB
:1005F00003AD039503AF469A00E002AB01E003AB05
:100600000EBD08E809BF01E000938A0004E20093F0
:100610007D0002E302AF78941EC049E145AB0019AA
:100620001109220933098FD0C4D0820193018BD0E4
:10063000DC011896ACD0ADD091D0429B04C0A8E2AA
:10064000B2E0A5D08BD004E8AFD000E093D004ECAA
:10065000ABD001E08FD000916A02002309F4FBDEE9
:1006600000916402002329F100916A02002319F02D
:10067000FC010A9502AF00E00093640202B718B7CC
:1006800011FF03C002E008BF0FEF10E012BF429B52
:1006900007C0043170F4979808B1087F08B904C006
:1006A000093238F0979A429A01E00093630210935E
:1006B000620209B70F7709BF00916302002359F462
:1006C000FC0104A515A5063920E0104020F001E04A
:1006D00003AB24A725A709B7006809BF00916302EF
:1006E000023009F0B8CFFC0166A177A104A115A1E1
:1006F000048F158F668F778F008C118C228C338C32
:10070000268D378D008F118F228F338F4488558827
:10071000668877884089518962897389441A550AA5
:10072000660A770A4489558966897789408B518B97
:10073000628B738B40E043AB42A9442309F06DCF39
:1007400001E002AB88CF0C94E00400871187228778
:10075000338744875587668777870895FC0105D0DE
:1007600044835583668377830895008311832283AE
:10077000338308950A93FC010081118101D034CDA7
:1007800022813381448155816681778108950C945B
:100790002E06DE010C94A606088119812A813B8170
:1007A0004C815D816E810895EBDC07E00A9308952A
:1007B000EEDF088319832A833B834C835D836E833A
:1007C0007F83089500008895FECF0FEA0DBF01E0FA
:1007D0000EBFC0E5D1E00E947407002311F00E9413
:1007E00084070E94D9020E94E2030C94E2034A9516
:1007F0002AF03695279517950795F9CF08953095E6
:100800002095109501951F4F2F4F3F4F08957A92D5
:100810006A925A924A92BA93AA939A938A930895A3
:100820007F806E805D804C80BB81AA8199818881A8
:10083000F0E0EC0FFD1FEF01089527973A932A93FC
:100840001A930A934A930D903D91FD91ED910D916C
:100850001D912D911C9017973324222443E0110CF5
:1008600037941694000C331FFF1FEE1F001F111F3B
:10087000221F111C221C4A95A9F7220F111C221CB1
:1008800014162406089411F48894139427952B8742
:100890001A870987E887FF833E830D824991099172
:1008A0001991299139910024EE27F3E0770F0794ED
:1008B0007695000F111F221F331F441F551F661FFF
:1008C000771FEE1FFA95A9F7660F771FEE1F7F17A8
:1008D000EF07089411F4889471E06795089567FD17
:1008E0001AC0000F111F221F331F441F551F661F00
:1008F0007150E040FF277130EF0769F084F766958B
:1009000057954795379527951795079508F4689457
:100910007F5FEF4FF0CFF7E0F023F43021F42EF0BB
:1009200003FD03C00BC008F409C0085F1F4F2F4F21
:100930003F4F4F4F5F4F6F4F7F4FEF4FFF2772304B
:10094000EF0718F467FF772709C0F7E07F3FEF074D
:1009500028F06627552744279A018A01F3E0660F9D
:10096000E69577956795E6957795679557954795B9
:100970003795279517950795FA95A9F7700D08955E
:100980007FE7702960EF552744279A018A0108956F
:10099000702D70786627F7CF7FEF6FEF08950024F2
:1009A00037FB07F816F40E94FF03412F522F632FE5
:1009B000302F002711272227E4E07EE1E8949ACF28
:1009C0000024F3CF70DF7F5FE34080F011247F319C
:1009D000E10570F007FC05C03FE72FEF1FEF0FEFB9
:1009E000089530E822271127002708953327FACFEA
:1009F000252F142F032F362F472F4F5141950E943B
:100A0000F70307FE08950C94FF03072EE62FEE0F61
:100A1000001CFFEFE03E0F0650F4E029E52BE42B2D
:100A2000E32BE22BE12BE02B8894B8940895E05E51
:100A3000E52BE42BE32BE22BE12BE02B19F00894C0
:100A4000B8940895889498943894089517960C90C3
:100A5000EE91EE0F001CFFEFE03E0F0680F4E02960
:100A60003E902E901E90E329E229E1293E902E909F
:100A70001E90E329E229E1298894B8940895E05E64
:100A80003E902E901E90E329E229E1293E902E907F
:100A90001E90E329E229E129A9F2D1CF7FEF6FEF80
:100AA0000895D4DF13F0D0F308951796FC911797AB
:100AB000F727A2F30895CADF51F00D911D912D91F2
:100AC0003D914D915D916D917C9117970895179689
:100AD000EC9117977E23089517967C91179752CF24
:100AE000089593DFD8F2EBF231F3B0DFB8F2A3F35D
:100AF000B9F32397E894A1DE17162E0638F50F8276
:100B0000E88779877119E209EE23E1F49F93BF9397
:100B10003F92972F7991E991F99109901990299035
:100B200039903694279417940794F795E79577951D
:100B300008F468949A95A9F79F91B8819B27BF9173
:100B40009F911EC0710DE21D2A9608CF17162E0622
:100B500061F06695579547953795279517950795B1
:100B600008F468947F5FEF4FF1CF30240F82E8875D
:100B700079877991E991F9910990199029903990A3
:100B8000AAF0070F1E1F2F1F301D411D521D631D90
:100B90000990E9917991C0F56795579547953795F3
:100BA0002795179507957F5FEF4FA4CE07171E0770
:100BB0002F073005410552056305B9F0C8F40EF062
:100BC0008894700BE10BF20B030A140A250A360A0B
:100BD000072F1E2F2F2F302D412D522D632D0990C1
:100BE000E9917991F0E80F2685CE77272396D2CE2A
:100BF0000EF40894070B1E0B2F0B30094109520904
:100C000063090990E991799175CEF0E87F2769CF62
:100C10001DDF38F031F01796FC911797F0787F2799
:100C200008953CCF13DFE8F3E3F31796FC91179791
:100C3000F0787F2708951796FC9117977F27707893
:100C40007158A0CE1796FC9117977F277078A2CE87
:100C50002A96702DF5CF2A96702D9CCED6DE08F3FD
:100C6000BBF201F3F3DEE8F233F361F32397E89488
:100C7000E4DD0324710DE21D7F5FE340FFEF7D3C67
:100C8000EF074CF3F7E07F3FEF0714F70F82E88799
:100C90007987AF93BF939F938F934F92F7E022246E
:100CA00011240024C001D001E8E0332477274990C3
:100CB00040FE08C0800FA11FB21F931F041E151E07
:100CC000261E371E000F111F221F331F441F551FE2
:100CD000661F771F4694EA9559F7882309F06894B0
:100CE000FA9579F08A2FAB2FB92F902D012C122C69
:100CF000232C012F122F232F342F452F562F672FF0
:100D0000D3CF632D522D412D302D292F8D010990E8
:100D1000E991799167FF03C07F5FEF4F07C0000F34
:100D2000111F221F331F441F551F661F4F908F91A5
:100D30009F91BF91AF91DECD89DE10F00BF06BCFAC
:100D4000ADCE84DEE9F3E0F37DCF75CF5EDEC0F398
:100D50009BF3B9F37BDEA0F3BBF3B9F32397E894DD
:100D60006CDD032467FD0AC0000F111F221F331F13
:100D7000441F551F661F7150E040F4CF3E8037FC82
:100D800019C0F881FF0FF883F981FF1FF983FA81F9
:100D9000FF1FFA83FB81FF1FFB83FC81FF1FFC8386
:100DA000FD81FF1FFD83331C3E82F1E01F1AF0E03E
:100DB0002F0AE4CF7150EC4F7119E2092AF4FFEFCA
:100DC0007D3CEF0708F447CFF7E07F3FEF070CF0DB
:100DD0003FCF0F82E88779879F93BF93AF93799135
:100DE000E991F99109901990299039906695579554
:100DF0004795379527951795079536942794179417
:100E00000794F795E7957795A7E09927B8E0990FAC
:100E100007171E072F07300541055205630540F0EF
:100E2000071B1E0B2F0B30094109520963099395CB
:100E3000000F111F221F331F441F551F661FBA9535
:100E400031F79A93AA9509F70A171A072A073A075A
:100E50004A075A076A0709F06894AF91BF919F91BA
:100E60000991199129913991499159916991099063
:100E7000E99179913FCDEADD59F11796FC911797E9
:100E8000FF2332F108940895E1DD10F1BEDD00F199
:100E900091F3E72F1796FC91EF271AF41797F7179E
:100EA00008953E902E901E901497411552056305AB
:100EB0007F0758F051F414963E902E901E900E909D
:100EC000001511052205330571F0772362F450F403
:100ED00088940895BBDDE0F398DDD0F3D9DFC0F34B
:100EE000089408950894089501E0089520E006D03C
:100EF000E9F70895259102D0E9F708952D9301505F
:100F00001040202F212B08958CE39FE0FC010591D8
:100F10001491FC013296A591B491FC01349625916F
:100F20003491422F432B19F0F901E4DF01C0DEDFD9
:100F300006961FE08834910748F308958000B001B9
:100F4000480F750030020000462E3A00502E3A003D
:100F500047487A004D487A006B487A00487A20006A
:100F60006D487A0073656B006D7320007573200007
:100F70006E73200070732000FCA9F1D24D62503FC7
:100F80000000000000408F40000000000000F03F23
:100F900000000000000024409A9999999999B93F5E
:100FA0008DEDB5A0F7C6A03E0000000080846EC1A4
:100FB00000000000000034400000000080846E410A
:080FC000000000000000704079
:00000001FF
:00000001FF
